:02000000BD2C15
:08000800FF00030E8312031335
:10001000B4000A0EB500040EB6008A110A12E52CCF
:10002000D208031D14280800F930FF3E031D1528CF
:100030000000D20B1428080000000000000000009F
:10004000000000000000D60B1C2808000330D40775
:10005000D40CD40C7F30D4050000D40B2C2808001D
:10006000D901DA01DC01DD01DB015B1A08000310B4
:10007000DC0DDD0DD30DD40DD90DDA0D56085A0265
:10008000031D442855085902031C4D285508D90260
:100090005608031CDA03DA025C14DB0A3528D101A6
:1000A000500851020318080064000130D2001020EB
:1000B000D10A5028831603178C185A288312031369
:1000C000520803178D000313540803178C0083167E
:1000D0008C130C1580300B0583120313D5008B1382
:1000E0005530831603178D00AA308D008C148C18A0
:1000F000772883120313D50803197F288B178316DB
:1001000003170C110800D201500803178D00831645
:100110008C130C1483120C080313D2005208D30062
:100120000800061086100611861106128612530E5C
:100130000F39D5000F30D50555180614D51886147B
:1001400055190615D5198615D408031D06160A304B
:10015000D6001C2086160A30D6001C2086120F30CE
:100160005305D5000A30D6001C2006108610061153
:1001700086110612861255180614D51886145519BC
:100180000615D5198615D408031D06160A30D600A3
:100190001C2086160A30D6001C2086120A30D60093
:1001A0001C200800D201D501D6014E08D300D4018D
:1001B000D21908004F1CE2285308D5070318D60AA5
:1001C0005408D607CF0C0310D30DD40DD20AD8286B
:1001D00004301F049F001F19EB28D00803190429BD
:1001E0001E08D100D201D10DD20DD10DD20DFC309F
:1001F000D10583161E0C8312D300D30CD30E03300B
:100200005305D104D20807291E08D100D201510894
:10021000D3005208D40008005008003A031D2029DA
:100220000130CD000030BE008530BD00D208031D76
:100230001D290E3083169F002029053083169F004C
:1002400083125108033C0318272983161F178313B1
:1002500083123E1883173D0884000008CC004D0827
:100260004C04D40080005108D400D501D40DD50D24
:10027000D40DD50DD40DD50DD40DD50DD40DD50D72
:10028000D40DD50DC03054050138D7005008D60024
:10029000D60DD60DD60DF830560557049F005308DD
:1002A000D400262008008313831203133E188317FB
:1002B0003D0884004C088000073083169F0083129D
:1002C0009F010800FF3083120313CF008316071726
:1002D000403083120705CF004F08D0000800FF30E0
:1002E00083120313CF00831687162030831207056D
:1002F000CF004F08D0000800FF3083120313CF0057
:1003000083160716103083120705CF004F08D00060
:1003100008008316031306138312061308008316BE
:1003200003130613831206170800CF1FA4292D30CC
:10033000D3001030D40091204E08003CD300CF09E8
:100340000318CF0A5308CE004E08D0004F08D10042
:1003500027304F02031DAE2910304E02031CDC294A
:10036000CF1BDC29D7015008D3005108D400D11F7E
:10037000BF29D309D409D30A0319D40AD70A1030E4
:10038000D5002730D60030205C08D200571CCA297F
:10039000D209D20A5208303ED3001030D400912046
:1003A0005208003C0318DC291030D0022730031C0F
:1003B0002830D102D203D02903304F02031DE22995
:1003C000E8304E02031C122ACF1B122AD801500813
:1003D000D3005108D400D11FF329D309D409D30A7B
:1003E0000319D40AD80AE830D5000330D6003020EB
:1003F0005C08D700581CFE29D709D70A5708D20035
:100400005208303ED3001030D40091205208003CF6
:100410000318122AE830D0020330031C0430D10242
:10042000D203062A4F08803AD30080305302031DBE
:100430001B2A64304E02031C472AD8015008D300FF
:100440005108D400D11F2A2AD309D409D30A031989
:10045000D40AD80A6430D500D60130205C08D70011
:10046000581C342AD709D70A5708D2005208303E00
:10047000D3001030D40091205208003C0318472AC2
:100480006430D002D108031CD103D2033C2A4F08A8
:10049000803AD30080305302031D502A0A304E02A6
:1004A000031C7C2AD8015008D3005108D400D11F66
:1004B0005F2AD309D409D30A0319D40AD80A0A3007
:1004C000D500D60130205C08D700581C692AD7090E
:1004D000D70A5708D2005208303ED3001030D4005B
:1004E00091205208003C03187C2A0A30D002D1081F
:1004F000031CD103D203712A5008303ED3001030C0
:10050000D400912008004E08D3001030D400912070
:100510000800CF08031D8F2A8030CF00912AC030F9
:10052000CF004E084F07D300D40191200230D000F5
:100530004F2008004E08D2004F08D3005008D400C6
:100540005A2008004E08D0004F08D10083205308DD
:10055000D000D10108008312031348083902CE00ED
:100560003A08CF00031CCF03CE0A0319CF0A4F0865
:100570003C02031DBD2A4E083B02031C8F213A0892
:100580003C02031DC52A39083B02031889210800D3
:100590007C21CE01D008031D4E14CB104E08031D44
:1005A000CB14CE01CF01A2225008C9000230CE00E8
:1005B000CF01A2225008CA004908CE000A30CF005D
:1005C000D2205508B9005608BA004A08B9070318DE
:1005D000BA0ACB1C232BB908BA08B90A0319BA0AFC
:1005E0003908E93A033003193A06031DFB2AE830BB
:1005F000B9000330BA00C830D20010203908D30047
:100600003A08D4000A30D500D60130205C08C90071
:100610004908CE000A30CF00D2205508D000560835
:10062000D10050083902CA00CE01CF014908D000DC
:10063000D1019A22023083120313CE00CF014A085F
:10064000D000D1019A226F21CE01D008031D4E1493
:100650004B114E08031D4B154B1D652B0130B90284
:10066000BA08031CBA033A08073C031D392B3908A2
:10067000D03C03183D2BB901BA01C830D20010207C
:100680003908D3003A08D4000A30D500D60130200A
:100690005C08C9004908CE000A30CF00D2205508B6
:1006A000D0005608D10050083902CA00CE01CF014F
:1006B0004908D000D1019A22023083120313CE00E0
:1006C000CF014A08D000D1019A2283120313CE0130
:1006D0000130CF0089225230CE0083226530CE0017
:1006E00083226730CE0083223D30CE00832220302B
:1006F000CE0083223908CE003A08CF009521203061
:10070000CE0083224330CE0083222030CE008322CD
:100710006730CE0083223D30CE0083222030CE00D1
:1007200083224808CE00CF0195212030CE008322BD
:100730002030CE0083222030CE0083222030CE0015
:1007400083222030CE00832208000130831203135D
:10075000CE00CF01A2225008C8006221CE01D008ED
:10076000031D4E144B104E08031D4B144B1CC42B81
:10077000C830D2001020480AC8000130CE00CF0196
:100780004808D000D1019A228312031348080A3C7A
:10079000031808000130C800CE00CF014808D0007F
:1007A000D1019A22080083120313CE01CF01A222A5
:1007B0005008C9000230CE00CF01A2225008CA0062
:1007C0004908CE000A30CF00D2205508B90056089B
:1007D000BA004A08B9070318BA0A3A08033C031DCD
:1007E000F32B3908E83C0318FB2BCE01CF01323044
:1007F000D000D1019A22013083120313CE00CF0121
:10080000A2225008C80048080A3C0318080001301A
:10081000CE00CF010130D000D1019A22080083160A
:100820000313061083120610831686108312861097
:100830008316061183120611831686118312861100
:1008400083160612831206128316861283128612EC
:100850000C30D0004F203330D300D401912002302F
:10086000D0004F203330D300D40191200230D0008B
:100870004F203230D300D40191200230D0004F20DD
:100880002C30D300D40191200230D0004F2006300C
:10089000D300D40191200230D0004F200C30D3007F
:1008A000D40191200230D0004F200130D300D40178
:1008B00091200230D0004F200230D300D40191208B
:1008C0000230D0004F20080083120313D001033000
:1008D000D100D2012830D3000C210130D000E82013
:1008E0005308CE005408CF0053214E08D0004F08C3
:1008F000D10008000730831603139F00C030810029
:100900000F24D32364245008BB005108BC00CE013F
:10091000CF0189222030CE0083222030CE008322D6
:100920005430CE0083226530CE0083226D30CE005D
:1009300083227030CE0083222030CE0083223D30CF
:10094000CE0083222030CE0083223B08CE003C081C
:10095000CF0095212030CE0083224330CE00832269
:100960002030CE0083222030CE0083222030CE00E3
:100970008322C822A523AB22822CD53083120313F5
:10098000A000C430A100BB30A200DC30A300A40151
:10099000A501A601A701A801A901AA01AB01AC010B
:1009A000AD01AE01AF01C201C301B701B801C4017D
:1009B000C501C601C701B001B101B201B301C00157
:1009C000C101BF018A110A127A2C83120313360E59
:1009D0008400350E8A00340E8300FF0E7F0E09005E
:02400E00313F40
:00000001FF
